:020000040000FA
:0400000000EF3CF0E1
:0477FC000000000089
:10780000A5EF3FF000C0E5FF01C0E5FF00EE62F02C
:10781000FAEC3EF0006E00C0F3F000C0F4F0FAECB9
:107820003EF0006E0001E96F00500001F427FAEC11
:107830003EF0006E0001E86F00500001F427FAEC02
:107840003EF0006E00C0F5F000500001F42700018A
:10785000F551040A24E10001E951D8A4DBD0E85134
:10786000D8A4D8D00001F351020A01E0D3D0FAEC39
:107870003EF0006E0001EB6F00500001F427FAECBF
:107880003EF0006E0001EA6F00500001F427FAECB0
:107890003EF0006E0001F427F451D8A4B3D00001EB
:1078A000F551010A20E1FAEC3EF0006E0001F427E8
:1078B000F451D8A4A7D00001F2B3B9EC3DF090EC9C
:1078C0003FF00001F2A50BD0C00E0001E46F770E6F
:1078D000E56FE66BE76BB9EC3DF090EC3FF0590ECD
:1078E00068EC3FF09AD00001EB510001E71914E178
:1078F0000001EA510001E6190FE10001E951000120
:10790000E5190AE1C00E0001E815006EC00E000185
:10791000E415016E00180FE00001F2A302D0B9ECEB
:107920003DF090EC3FF0E8C0E4F0E9C0E5F0EAC0DB
:10793000E6F0EBC0E7F00001F551040A01E15ED08A
:107940000001F551D8A462D00001F351D8B456D04B
:107950000001EB51D8A45AD0EA51E00BD8A456D07C
:107960000001F2A912D00001F35142EC3EF0400EAA
:107970009BEC3FF00001E95142EC3EF00001E85180
:1079800042EC3EF0200E9BEC3FF0EAC0F8FFE9C06D
:10799000F7FFE8C0F6FF000100EE6AF022EE00F00B
:1079A000E8513F0BD926D8B0DA2ADD52FAEC3EF086
:1079B0000001F427DC6E0900F55C05E00001F283AC
:1079C0002A0E9BEC3FF00001F2A906D0DF5042ECFA
:1079D0003EF0200E9BEC3FF00001F32FE7D7FAECCE
:1079E0003EF0006E0001F427F45108E00001E46964
:1079F000E569E669E7690001F29304D0580E68EC86
:107A00003FF00BD07A0E68EC3FF007D0750E68ECB3
:107A10003FF003D06C0E68EC3FF0E4CF01F0E4CF10
:107A200000F01200FF0E926E936E946E966ED0EC84
:107A30003FF0970ED56E8B8A949AB06A3F0EAF6E68
:107A4000B886AC8AAC84AC8CAC90AB8CAB8E0001AD
:107A5000E46BE56BE66BE76B0001E86BE96BEA6BE7
:107A6000EB6B90EC3FF00001F26B93988A888B9A55
:107A7000AB984B0E9BEC3FF0AFEC3FF00001EC6B92
:107A8000ED6B8BBA02D0AFEC3FF00001606BBAEC4B
:107A90003EF000016051D8B45CD08B9AAB988AA8B4
:107AA00002D08A9801D08A8861C000F00050520A42
:107AB00003E159EC3FF00BD00050500A03E14AECCF
:107AC0003FF005D00050560A02E176EC3EF000018E
:107AD000F2A13FD00050450A03E138EC3FF039D025
:107AE00000503A0A03E102EC3CF033D00050720A35
:107AF00003E199EC3EF02DD00050410A03E1D3ECB4
:107B00003FF027D00050760A24E1006A000162515C
:107B1000300A01E1002A0050D880E866D890006A57
:107B200000360050010BE838E840F46E0001F251D5
:107B3000F70BF410F26F320E0001625D006A00363E
:107B40000050010BE838F46E0001F251EF0BF41015
:107B5000F26F0001F2B195D70001ED51800F800F57
:107B600002E1A10EEC5DD8A08CD7D3EC3FF089D711
:107B7000120000C0E5FF01C0E5FF02C0E5FF03C041
:107B8000E5FF0001E4513F0B04E0210E9BEC3FF0C8
:107B900070D00001E75103E1E651E00BD8A469D0B1
:107BA000780E0001E55D02E1000EE45D01E361D0C5
:107BB000E4C000F0E5C001F0E6C002F0E7C003F069
:107BC000005001100210031013E100C2E0F001C2E6
:107BD000E1F002C2E2F003C2E3F00201006BEF0E3B
:107BE000016F3C0E026FF00E036F0001F28515D09D
:107BF0000050C00A07E10150770A04E1025002E197
:107C0000035001E00AD0E0C03CF2E1C03DF2E2C026
:107C10003EF2E3C03FF20001F2950001F2A70BD063
:107C2000200E9BEC3FF00001E55142EC3EF00001DC
:107C3000E45142EC3EF0E6C0F8FFE5C0F7FFE4C0D7
:107C4000F6FF940EB7EC3FF00A0002EE00F00001E0
:107C5000080EEE6F080EEF6FEE50F56E0F00EF2F6F
:107C6000FBD7840E84D9EE2FF5D7A694570E68EC77
:107C70003FF0E4CF03F0E4CF02F0E4CF01F0E4CF33
:107C800000F0120000C0E5FF01C0E5FF02C0E5FF03
:107C9000006E00380F0B026E300E02260250016E8D
:107CA0003A0E015C06E30150026E070E02260250F6
:107CB000016E01509BEC3FF00F0E0014006E300E71
:107CC00000260050016E3A0E015C06E30150006E82
:107CD000070E00260050016E01509BEC3FF0E4CFF0
:107CE00002F0E4CF01F0E4CF00F0120000EE62F009
:107CF000000160050001EF6FEF07010EEE6FEE511E
:107D0000CAEC3FF004E10A0EEE6FCAEC3FF0EE5C05
:107D1000D8A41200EE2BEF2FF2D7EE51CAEC3FF0B1
:107D2000D8A41200560E68EC3FF00001F281F295E3
:107D3000120000C0E5FF00EE62F0FAEC3EF0F76ED4
:107D4000FAEC3EF0F66E720E9BEC3FF0200E9BECD0
:107D50003FF0100E006E0900F55042EC3EF0200E90
:107D60009BEC3FF0002EF7D70A0E9BEC3FF0E4CFE0
:107D700000F01200C4EC3FF0000100EE60F0DAEC1D
:107D80003EF0E86614D0AE50EE6EEE6FEF6FD8B4F2
:107D90000ED0C4EC3FF0DAEC3EF0E86608D0AE500E
:107DA000EE6EEF27EE2FF5D7EF53D8B41200000197
:107DB000606B12009EBA08D0F2A4FCD70001EC2B35
:107DC00001E3ED2BE86815D08A98ABB202D0ABA4E2
:107DD00004D0AFEC3FF0E8680CD0ABA009D0AE50B7
:107DE00005E1C4EC3FF0DAEC3EF003D0D3EC3FF019
:107DF000E86A12000001EECFEEF0EECFEFF0D00E09
:107E0000EE27EF27F60EEE25F90ED8B0EE27F60E88
:107E1000EF25F90ED8B0EF27EE39EF25E850120024
:107E200000EE68F000016051F80F0001EE6F09E00C
:107E3000F05D07E3EE50A86E84EC3FF0A92AEE2F28
:107E4000F9D7A86A84EC3FF0120000C0E5FF01C03A
:107E5000E5FF006A00EE62F0060E016EEE500026AD
:107E6000012EFCD70050E4CF01F0E4CF00F0120067
:107E700000EE61F0000160510001EE6F07E0EE07D7
:107E800005E0EE509BEC3FF0EE2FFBD70A0E9BEC8B
:107E90003FF0120025EC3FF0B80A0AE1010EA96E8E
:107EA000080E0001F06F10EC3FF0500E68EC3FF050
:107EB000120025EC3FF0A00A0AE10A0EA96E100E8E
:107EC0000001F06F10EC3FF0520E68EC3FF0120032
:107ED00000C0E5FF006E200E9BEC3FF000509BECD5
:107EE0003FF00A0E9BEC3FF0E4CF00F01200700E62
:107EF000D36E9B8C0F013A9FFF0E92689368946833
:107F00009668626AF19E1200A69EA69CA684550EF3
:107F1000A76EAA0EA76EA682A6B2FED7A6941200DE
:107F20000001F2930001400EEE6F02EE00F0EE68E9
:107F3000EE2FFDD7120000C0E5FF006E9EA8FED711
:107F400000C0ADFFE4CF00F0120011EEFFF021EE13
:107F5000FFF0F86AA68EA69C12EC3DF0FFD7ACA20B
:107F6000FED78B8AAE50AE50AB98AB881200A66E8F
:107F7000550EA76EAA0EA76EA6821200C0EF3FF0A4
:107F800012EC3DF0C2EF3FF0F70ED76EF80ED66E52
:107F9000F2941200A96EA69CA69EA680A85012007C
:0A7FA00077EC3FF01200FEEF3BF01B
:020000040030CA
:0E000000FF38FAE2FF6FBBFFFFFFFFFFFFFFBD
:0200000400F00A
:0400000000000000FC
:00000001FF
